:020000040000fa
:08000000407f04000000000035
:020000040000fa
:1002000000000000000000000000000000000000ee
:1002100000000000000000000000000000000000de
:1002200000000000000000000000000000000000ce
:1002300000000000000000000000000000000000be
:10fe8000cf88200060ff20000001880000000000f3
:10fe900000002800601088000040200070108800da
:10fea000f0002000a0108800048020002f00070030
:10feb000114cb1003a003a0052c7b30082108800da
:10fec000b2c4b300821088008006eb0004802000da
:10fed00046002000250007000603e900fdff3a0068
:10fee0000c4080001340800093018800160620001b
:10fef0001e0007000603e900fdff3a000d00e000c8
:10ff000003003200e2c4b30082108800eeff370025
:10ff1000000ebb00100424000060fe000a00070071
:10ff2000448020001f00080003000000345ebb0076
:10ff30003456bb0034cebb000c86e8001000240011
:10ff400001000700deff3700003b8800500520005d
:10ff5000303b8800a00a2000303b880061e7a80001
:10ff60000000000000000000000006005a00200011
:10ff70000b0020000e02ae0004003700911080003c
:10ff8000015a78008dc64000000006000060fe00a7
:10ff90008b05e900f7ff3a000a05e900f4ff3a0093
:08ffa0000c22ef00b2ff370054
:020000040000fa
:10ffa800000800008c0000000000000000000000b5
:020000040000fa
:0200000401f009
:0400000002c3000037
:020000040000fa
:0200000401f009
:04000400ff7f00007a
:020000040000fa
:0200000401f009
:040008007fff000076
:020000040000fa
:0200000401f009
:04001400ffff0000ea
:020000040000fa
:10000800dc7f0000dc7f0000dc7f0000dc7f00007c
:10001800dc7f0000dc7f0000dc7f0000dc7f00006c
:10002800dc7f0000dc7f0000dc7f0000dc7f00005c
:10003800dc7f0000dc7f0000dc7f0000dc7f00004c
:10004800dc7f0000dc7f0000dc7f0000dc7f00003c
:10005800dc7f0000dc7f0000dc7f0000dc7f00002c
:10006800dc7f0000dc7f0000dc7f0000dc7f00001c
:10007800dc7f0000dc7f0000dc7f0000dc7f00000c
:10008800dc7f0000dc7f0000dc7f0000dc7f0000fc
:10009800dc7f0000dc7f0000dc7f0000dc7f0000ec
:1000a800dc7f0000dc7f0000dc7f0000dc7f0000dc
:1000b800dc7f0000dc7f0000dc7f0000dc7f0000cc
:1000c800dc7f0000dc7f0000dc7f0000dc7f0000bc
:1000d800dc7f0000dc7f0000dc7f0000dc7f0000ac
:1000e800dc7f0000dc7f0000dc7f0000dc7f00009c
:0800f800dc7f0000dc7f00004a
:020000040000fa
:10010800dc7f0000dc7f0000dc7f0000dc7f00007b
:10011800dc7f0000dc7f0000dc7f0000dc7f00006b
:10012800dc7f0000dc7f0000dc7f0000dc7f00005b
:10013800dc7f0000dc7f0000dc7f0000dc7f00004b
:10014800dc7f0000dc7f0000dc7f0000dc7f00003b
:10015800dc7f0000dc7f0000dc7f0000dc7f00002b
:10016800dc7f0000dc7f0000dc7f0000dc7f00001b
:10017800dc7f0000dc7f0000dc7f0000dc7f00000b
:10018800dc7f0000dc7f0000dc7f0000dc7f0000fb
:10019800dc7f0000dc7f0000dc7f0000dc7f0000eb
:1001a800dc7f0000dc7f0000dc7f0000dc7f0000db
:1001b800dc7f0000dc7f0000dc7f0000dc7f0000cb
:1001c800dc7f0000dc7f0000dc7f0000dc7f0000bb
:1001d800dc7f0000dc7f0000dc7f0000dc7f0000ab
:1001e800dc7f0000dc7f0000dc7f0000dc7f00009b
:0801f800dc7f0000dc7f000049
:020000040000fa
:04ffb8000000fe0047
:00000001FF
